BL51 BANKED LINKER/LOCATER V5.03                                                        10/31/2008  13:27:12  PAGE 1


BL51 BANKED LINKER/LOCATER V5.03, INVOKED BY:
C:\KEIL\C51\BIN\BL51.EXE .\OUT\SyncMOS.obj, .\OUT\main.obj, .\OUT\SM_EEPROM.obj, .\OUT\Gotoisp_59D.obj TO .\OUT\SyncmOS 
>> eeprom PRINT (.\LST\SyncmOS eeprom.m51) RAMSIZE (256)


MEMORY MODEL: SMALL


INPUT MODULES INCLUDED:
  .\OUT\SyncMOS.obj (?C_STARTUP)
  .\OUT\main.obj (MAIN)
  .\OUT\SM_EEPROM.obj (SM_EEPROM)
  .\OUT\Gotoisp_59D.obj (GOTOISP_59D)
  C:\KEIL\C51\LIB\C51S.LIB (?C_INIT)


LINK MAP OF MODULE:  .\OUT\SyncmOS eeprom (?C_STARTUP)


            TYPE    BASE      LENGTH    RELOCATION   SEGMENT NAME
            -----------------------------------------------------

            * * * * * * *   D A T A   M E M O R Y   * * * * * * *
            REG     0000H     0008H     ABSOLUTE     "REG BANK 0"
            DATA    0008H     0002H     UNIT         _DATA_GROUP_
            IDATA   000AH     0074H     UNIT         ?ID?MAIN
            IDATA   007EH     0001H     UNIT         ?STACK

            * * * * * * *   C O D E   M E M O R Y   * * * * * * *
            CODE    0000H     0003H     ABSOLUTE     
            CODE    0003H     008FH     UNIT         ?C_C51STARTUP
            CODE    0092H     0059H     UNIT         ?PR?MAIN?MAIN
            CODE    00EBH     003EH     UNIT         ?C_INITSEG
            CODE    0129H     001EH     UNIT         ?PR?_ISP_PROGRAM_BYTE?SM_EEPROM
            CODE    0147H     001BH     UNIT         ?PR?READ?MAIN
            CODE    0162H     001BH     UNIT         ?PR?WRITE?MAIN
            CODE    017DH     0015H     UNIT         ?PR?_DELAY2?MAIN
            CODE    0192H     0013H     UNIT         ?PR?_ISP_ERASE_SECTOR?SM_EEPROM
            CODE    01A5H     000FH     UNIT         ?PR?EEPROM_ENABLE?SM_EEPROM
            CODE    01B4H     000EH     UNIT         ?PR?_ISP_READ_BYTE?SM_EEPROM
            CODE    01C2H     0006H     UNIT         ?PR?EEPROM_DISABLE?SM_EEPROM
            CODE    01C8H     0003H     UNIT         ?PR?GOTOISP_59D?GOTOISP_59D



OVERLAY MAP OF MODULE:   .\OUT\SyncmOS eeprom (?C_STARTUP)


SEGMENT                                   DATA_GROUP 
  +--> CALLED SEGMENT                   START    LENGTH
-------------------------------------------------------
?C_C51STARTUP                           -----    -----
  +--> ?PR?MAIN?MAIN
  +--> ?C_INITSEG

?PR?MAIN?MAIN                           0008H    0001H
  +--> ?PR?GOTOISP_59D?GOTOISP_59D
  +--> ?PR?_ISP_ERASE_SECTOR?SM_EEPROM
BL51 BANKED LINKER/LOCATER V5.03                                                      10/31/2008  13:27:12  PAGE 2


  +--> ?PR?WRITE?MAIN
  +--> ?PR?READ?MAIN
  +--> ?PR?_DELAY2?MAIN

?PR?_ISP_ERASE_SECTOR?SM_EEPROM         -----    -----
  +--> ?PR?EEPROM_ENABLE?SM_EEPROM
  +--> ?PR?EEPROM_DISABLE?SM_EEPROM

?PR?WRITE?MAIN                          0009H    0001H
  +--> ?PR?_ISP_PROGRAM_BYTE?SM_EEPROM

?PR?_ISP_PROGRAM_BYTE?SM_EEPROM         -----    -----
  +--> ?PR?EEPROM_ENABLE?SM_EEPROM
  +--> ?PR?EEPROM_DISABLE?SM_EEPROM

?PR?READ?MAIN                           0009H    0001H
  +--> ?PR?_ISP_READ_BYTE?SM_EEPROM



SYMBOL TABLE OF MODULE:  .\OUT\SyncmOS eeprom (?C_STARTUP)

  VALUE           TYPE          NAME
  ----------------------------------

  -------         MODULE        ?C_STARTUP
  C:0003H         SEGMENT       ?C_C51STARTUP
  I:007EH         SEGMENT       ?STACK
  C:0000H         PUBLIC        ?C_STARTUP
  D:00E0H         SYMBOL        ACC
  D:00F0H         SYMBOL        B
  D:0083H         SYMBOL        DPH
  D:0082H         SYMBOL        DPL
  N:0000H         SYMBOL        IBPSTACK
  N:0100H         SYMBOL        IBPSTACKTOP
  N:0080H         SYMBOL        IDATALEN
  C:0009H         SYMBOL        IDATALOOP
  N:0000H         SYMBOL        PBPSTACK
  N:0000H         SYMBOL        PBPSTACKTOP
  N:0000H         SYMBOL        PDATALEN
  N:0000H         SYMBOL        PDATASTART
  N:0000H         SYMBOL        PPAGE
  N:0000H         SYMBOL        PPAGEENABLE
  D:00A0H         SYMBOL        PPAGE_SFR
  D:0081H         SYMBOL        SP
  C:0003H         SYMBOL        STARTUP1
  N:0000H         SYMBOL        XBPSTACK
  N:0000H         SYMBOL        XBPSTACKTOP
  N:0000H         SYMBOL        XDATALEN
  N:0000H         SYMBOL        XDATASTART
  C:0000H         LINE#         92
  C:0003H         LINE#         100
  C:0006H         LINE#         104
  C:0008H         LINE#         105
  C:0009H         LINE#         106
  C:000AH         LINE#         107
  C:000CH         LINE#         160
BL51 BANKED LINKER/LOCATER V5.03                                                      10/31/2008  13:27:12  PAGE 3


  C:000FH         LINE#         164
  -------         ENDMOD        ?C_STARTUP

  -------         MODULE        MAIN
  C:0000H         SYMBOL        _ICE_DUMMY_
  D:0080H         PUBLIC        P0
  D:0090H         PUBLIC        P1
  D:00A0H         PUBLIC        P2
  D:00B0H         PUBLIC        P3
  D:00D8H         PUBLIC        P4
  D:00B8H         PUBLIC        IP
  C:0147H         PUBLIC        read
  C:017DH         PUBLIC        _delay2
  C:0092H         PUBLIC        main
  C:0162H         PUBLIC        write
  B:0080H.0       PUBLIC        P00
  D:0098H         PUBLIC        SCON
  D:0088H         PUBLIC        TCON
  I:000AH         PUBLIC        data_buf
  I:0044H         PUBLIC        read_buf
  D:00BFH         PUBLIC        AUXR
  D:00A8H         PUBLIC        IER
  D:00C8H         PUBLIC        T2CON
  D:00D0H         PUBLIC        PSW
  -------         PROC          MAIN
  -------         DO            
  D:0008H         SYMBOL        m
  -------         ENDDO         
  C:0092H         LINE#         23
  C:0092H         LINE#         24
  C:0092H         LINE#         26
  C:0095H         LINE#         27
  C:0098H         LINE#         28
  C:0098H         LINE#         29
  C:009BH         LINE#         30
  C:009BH         LINE#         31
  C:00A0H         LINE#         32
  C:00A3H         LINE#         33
  C:00A6H         LINE#         36
  C:00A6H         LINE#         37
  C:00A6H         LINE#         38
  C:00A9H         LINE#         39
  C:00A9H         LINE#         40
  C:00B7H         LINE#         41
  C:00B7H         LINE#         42
  C:00BEH         LINE#         43
  C:00C1H         LINE#         44
  C:00C4H         LINE#         45
  C:00CCH         LINE#         46
  C:00D4H         LINE#         47
  C:00D6H         LINE#         49
  C:00D6H         LINE#         50
  C:00DDH         LINE#         51
  C:00E0H         LINE#         53
  -------         ENDPROC       MAIN
  -------         PROC          READ
  -------         DO            
BL51 BANKED LINKER/LOCATER V5.03                                                      10/31/2008  13:27:12  PAGE 4


  D:0009H         SYMBOL        m
  -------         ENDDO         
  C:0147H         LINE#         57
  C:0147H         LINE#         58
  C:0147H         LINE#         60
  C:014AH         LINE#         62
  C:0158H         LINE#         63
  C:0161H         LINE#         65
  -------         ENDPROC       READ
  -------         PROC          WRITE
  -------         DO            
  D:0009H         SYMBOL        m
  -------         ENDDO         
  C:0162H         LINE#         66
  C:0162H         LINE#         67
  C:0162H         LINE#         69
  C:0165H         LINE#         71
  C:0173H         LINE#         73
  C:017CH         LINE#         75
  -------         ENDPROC       WRITE
  -------         PROC          _DELAY2
  D:0006H         SYMBOL        x
  -------         DO            
  D:0005H         SYMBOL        y
  -------         ENDDO         
  C:017DH         LINE#         76
  C:017DH         LINE#         77
  C:017DH         LINE#         79
  C:0187H         LINE#         80
  C:0189H         LINE#         81
  C:018FH         LINE#         82
  C:0191H         LINE#         83
  C:0191H         LINE#         84
  -------         ENDPROC       _DELAY2
  -------         ENDMOD        MAIN

  -------         MODULE        SM_EEPROM
  C:0000H         SYMBOL        _ICE_DUMMY_
  D:0080H         PUBLIC        P0
  D:0090H         PUBLIC        P1
  D:00A0H         PUBLIC        P2
  D:00B0H         PUBLIC        P3
  D:00D8H         PUBLIC        P4
  B:00A8H.7       PUBLIC        EA
  C:0192H         PUBLIC        _isp_erase_sector
  D:00B8H         PUBLIC        IP
  C:0129H         PUBLIC        _isp_program_byte
  D:00F7H         PUBLIC        ISPC
  D:0098H         PUBLIC        SCON
  D:0088H         PUBLIC        TCON
  D:00F4H         PUBLIC        ISPFAH
  D:00F5H         PUBLIC        ISPFAL
  C:01B4H         PUBLIC        _isp_read_byte
  D:00E0H         PUBLIC        ACC
  D:00A8H         PUBLIC        IER
  C:01C2H         PUBLIC        EEPROM_Disable
  D:00C8H         PUBLIC        T2CON
BL51 BANKED LINKER/LOCATER V5.03                                                      10/31/2008  13:27:12  PAGE 5


  C:01A5H         PUBLIC        EEPROM_Enable
  D:00F6H         PUBLIC        ISPFD
  D:00D0H         PUBLIC        PSW
  D:00BFH         PUBLIC        SCONF
  -------         PROC          _ISP_READ_BYTE
  D:0006H         SYMBOL        add
  -------         DO            
  D:0082H         SYMBOL        tempP
  D:0007H         SYMBOL        rdata
  -------         ENDDO         
  C:01B4H         LINE#         11
  C:01B4H         LINE#         12
  C:01B4H         LINE#         16
  C:01BEH         LINE#         17
  C:01C1H         LINE#         18
  C:01C1H         LINE#         20
  -------         ENDPROC       _ISP_READ_BYTE
  -------         PROC          EEPROM_ENABLE
  C:01A5H         LINE#         25
  C:01A5H         LINE#         26
  C:01A5H         LINE#         27
  C:01A8H         LINE#         28
  C:01ABH         LINE#         29
  C:01AEH         LINE#         30
  C:01B1H         LINE#         31
  C:01B3H         LINE#         32
  -------         ENDPROC       EEPROM_ENABLE
  -------         PROC          EEPROM_DISABLE
  C:01C2H         LINE#         36
  C:01C2H         LINE#         37
  C:01C2H         LINE#         38
  C:01C5H         LINE#         39
  C:01C7H         LINE#         40
  -------         ENDPROC       EEPROM_DISABLE
  -------         PROC          _ISP_PROGRAM_BYTE
  D:0002H         SYMBOL        add
  D:0005H         SYMBOL        dat
  -------         DO            
  D:0007H         SYMBOL        addh
  D:0006H         SYMBOL        addl
  -------         ENDDO         
  C:0129H         LINE#         42
  C:012DH         LINE#         43
  C:012DH         LINE#         45
  C:0130H         LINE#         46
  C:0132H         LINE#         47
  C:0138H         LINE#         48
  C:0139H         LINE#         49
  C:013AH         LINE#         50
  C:013CH         LINE#         51
  C:013EH         LINE#         53
  C:0141H         LINE#         54
  C:0144H         LINE#         56
  C:0144H         LINE#         57
  -------         ENDPROC       _ISP_PROGRAM_BYTE
  -------         PROC          _ISP_ERASE_SECTOR
  D:0007H         SYMBOL        num
BL51 BANKED LINKER/LOCATER V5.03                                                      10/31/2008  13:27:12  PAGE 6


  -------         DO            
  D:0007H         SYMBOL        addh
  D:0006H         SYMBOL        addl
  -------         ENDDO         
  C:0192H         LINE#         60
  C:0192H         LINE#         61
  C:0192H         LINE#         64
  C:0194H         LINE#         65
  C:0197H         LINE#         67
  C:0197H         LINE#         68
  C:0197H         LINE#         69
  C:019AH         LINE#         70
  C:019CH         LINE#         72
  C:019FH         LINE#         73
  C:01A2H         LINE#         75
  C:01A2H         LINE#         76
  -------         ENDPROC       _ISP_ERASE_SECTOR
  -------         ENDMOD        SM_EEPROM

  -------         MODULE        GOTOISP_59D
  C:01C8H         SEGMENT       ?PR?GOTOISP_59D?GOTOISP_59D
  C:01C8H         PUBLIC        GOTOISP_59D
  C:01C8H         LINE#         11
  -------         ENDMOD        GOTOISP_59D

Program Size: data=127.0 xdata=0 code=459
LINK/LOCATE RUN COMPLETE.  0 WARNING(S),  0 ERROR(S)
